S1130030CE00C4BDE07EBDE047DF28DF24CE00D182
S1130040BDE07EBDE047DF2ABDC36396258BFF97E5
S113005027962489019726912A251026069627910A
S11300602B2508962A9726962B97278D1D862BBD20
S1130070E1D196244C9724912A25D02606962591E1
S11300802B25C8862FBDE1D120A65FDE24E7009C86
S11300902627030820F7DE24DF201743A70008DF04
S11300A022DE20A6004311261ADE22A60011261302
S11300B09C2626EADE20089C2626DDC1FF27035362
S11300C020C9393F0D0A00005354415254203D20A9
S11300D0042020454E44203D200413FD0000000070
S105A0480030E2
